:1000000000308A003C280000831A0A28A500030E4D
:10001000A6000F288312A500030EA600A6140A0846
:10002000AD008A018313A50E0408A7002008A800CC
:100030002108A9002208AA002308AB002408AC006C
:1000400083128C308400001C27280C1842282708B3
:1000500084002808A0002908A1002A08A2002B0873
:10006000A3002C08A4002D088A00260E830083120A
:10007000250EA61883160900FF2383169000003072
:100080008A00282BB70364000C108A1127288316D6
:10009000FF30900083120330B7008F018E01B5301E
:1000A000900083160C14C03083128B0483161F0833
:1000B000F03901389F0083121F1383161F08F0398F
:1000C00002389F0083121F1383161F08F039083867
:1000D0009F0083121F1383161F08F0399F0083129D
:1000E0001F1383161F080F3910389F0083121F0833
:1000F0000C3981389F000C30A1001F08C33921043E
:100100009F000D30A000073081018130840000087D
:10011000F0390738800064000008F03920048000BE
:100120008316051183120511831605168312412BC0
:10013000BA01BB01831685128312851283168515B9
:1001400083128519B628BA0A0319BB0A3A08FA3C81
:10015000031DB528BB08031DB5288316851283121D
:10016000851683168516D42883129E288316851536
:100170008312851DCE28BA0A0319BB0A3A08FA3C35
:10018000031DCD28BB08031DCD28831685128312BD
:10019000851683168516D4288312B62883168512F1
:1001A0008312851683168516831200340A30BE002A
:1001B0003A080039A0003B080239A30020082304B4
:1001C0000319E7288316851283128516EB288316F8
:1001D000851283128512BD01BC0183168515831219
:1001E00085190529BC0A0319BD0A3C087D3C031D7D
:1001F0000429BD08031D0429831685128312851660
:10020000831685162D298312ED280310BA0DBB0D18
:10021000BD01BC01831685158312851D2229BC0AE8
:100220000319BD0A3C087D3C031D2129BD08031D9F
:1002300021298316851283128516831685162D298A
:1002400083120A29BE0BD8280830A000A00B26294B
:100250008316851283128512831683120034BA0125
:10026000BB018316851283128516831685168312A9
:10027000BB01BA0183168515831285194A29BA0A6A
:100280000319BB0A3A08F43C031D49293B0B4929D1
:100290007A293A29831685168312851E51293C1026
:1002A00052293C14BB01BA01831685158312851DA2
:1002B0006429BA0A0319BB0A3A08F43C031D6329EE
:1002C0003B0B63297A295429BB01BA018316851691
:1002D0008312851A7629BA0A0319BB0A3A08F43C34
:1002E000031D75293B0B75297A29662900303C18B6
:1002F0000130A10000342F1C042BAF1C042B8316EB
:1003000085168312851A042B831685158312851D85
:10031000042BB901B801831685158312851DAC29FC
:10032000B80A0319B90A3808323C031DAB29B908C9
:10033000031DAB29831685168312851AA1292F1058
:10034000A2292F148316851583128519A929AF10A8
:10035000AA29AF14142B8B29B901B801831685156E
:1003600083128519CF29B80A0319B90A3808323C13
:10037000031DCE29B908031DCE29831685168312C5
:10038000851AC4292F10C5292F14831685158312A9
:100390008519CC29AF10CD29AF14142BAE298316A3
:1003A00085168312851AE529831685168312851A08
:1003B000DB292F10DC292F1483168515831285194C
:1003C000E329AF10E429AF14142BB901B801831647
:1003D00085158312851D042BB80A0319B90A8316E3
:1003E00085168312851AEB2A831685158312851DBF
:1003F000EB2ABB01BC01BD01BA013A08073C031C52
:10040000372ABD01BC01831685158312851D152A67
:10041000BC0A0319BD0A3C08F43C031D142A3D0B19
:10042000142A0030A100392A032ABD01BC01831619
:100430008515831285192A2ABC0A0319BD0A3C08AE
:100440007D3C031D292ABD08031D292A0030A10077
:10045000392A172A03103B0DBE008316851600307B
:100460008312851A01303E04BB00BA0AFD293B08FD
:10047000A1002108AE002E08B13C031DC22A2F1591
:100480009F149F18412A83161E088312B0001E086D
:10049000B1003108B5003008B4000030A1001F08D9
:1004A000C33921049F0098203108BB003008BA00EE
:1004B000D6209F149F185A2A83161E088312B00054
:1004C0001E08B1000430A1001F08C33921049F0099
:1004D0003008B4070318B50A3108B5072F21A10861
:1004E000031D792A0C30A1001F08C33921049F0085
:1004F000B02A3108BB003008BA00D6209F149F18DC
:100500007F2A83161E088312B0001E08B10030082F
:10051000B4070318B50A3108B5072F21A108031D38
:10052000982A0C30A1001F08C33921049F00B02A6B
:100530003108BB003008BA00D6202F213508BB0097
:100540003408BA00D62083168512831285168316C6
:1005500085160C308312A1001F08C33921049F00A7
:10056000831685168312851AB72A2F10B82A2F14DE
:100570008316851583128519BF2AAF10C02AAF14C0
:10058000142BEB2A2E08B23C031DEB2A9820BB014A
:100590000330BA00D6202F21A1080319DA2ABB01A3
:1005A0006930BA00D6208316851283128516831609
:1005B00085168312831685168312851AE12A2F1059
:1005C000E22A2F148316851583128519E92AAF10A4
:1005D000EA2AAF14142B3808323C031D032BB90848
:1005E000031D032B831685168312851AF92A2F10F3
:1005F000FA2A2F148316851583128519012BAF1043
:10060000022BAF14142BE729831685168312851A43
:100610000B2B2F100C2B2F14831685158312851985
:10062000132BAF10142BAF14462B38308400000866
:100630000319272B0130A100A001A00B1D2BA10B3A
:100640001C2B9E30A000A00B232B800B1A2B0034F8
:1006500084011F30830583161F08F0399F00831221
:100660001F1307309F00FF30B0000330B10020306F
:10067000B2000130B3002F11FA30B6000330B700DA
:10068000472883160511831205117B29B708031D1E
:10069000642B0330B700B60B642BFA30B600003081
:1006A0002F190130003A031D632B831605118312A5
:1006B00005150A30B800152383160511831205119C
:0C06C0000A30B80015232F11412B6300F5
:02400E00CC39AB
:00000001FF
